:0300000002277163
:0C27710078FFE4F6D8FD7581460227B819
:100F6C000A53746172743A20004950436F6E6E6577
:100F7C0063745245510A00444843502D4F4B0A00AC
:100F8C004950436F6E6E65637400C0E4E0EFF2E5A8
:100F9C00F020D1E8EDEAEEEC4950285243290A0042
:100FAC00C2E5F0F1E8FF20495020ECEEE4F3EBFF52
:100FBC003A20322E3420EEF22032302E31312E32C5
:100FCC003030350A00C4E0F2E020F1EEE7E4E0ED69
:100FDC00E8FF3A20004F6374203133203230303632
:100FEC0000200031313A34353A3232000A000A50CE
:100FFC00524F473A20202020202020202020202043
:10100C0020202020202020202020202020202020D4
:10101C0020202020202020202020202020202020C4
:10102C0020202020202020202020202020202020B4
:10103C002020202020202020200A0044756D70588C
:10104C00202020202030302030312030322030330E
:10105C0020303420303520303620303720303820C6
:10106C003039203041203042203043203044203071
:10107C00452030460A003A200044756D704420200B
:10108C0020202030302030312030322030332030BE
:10109C00342030352030362030372030382030396D
:1010AC002030412030422030432030442030452035
:1010BC0030460A00457272206B65790052642065D7
:1010CC006570726F6D0A005264204D454D0A0044E4
:1010DC00656275674950204F4E0A0044656275671A
:1010EC004950204F46460A00446562756755736542
:1010FC0072204F6E0A0044656275675573657220E5
:10110C004F46460A0044656275674D7367204F6E03
:10111C000A0044656275674D7367204F46460A00A6
:10112C00436F6E666967206C6F636B210A005772A0
:10113C0020656570726F6D0A0020536176652065BD
:10114C006570726F6D210A00457272204D4143210A
:10115C00004C6F61643E3E00576169745265737454
:10116C0061727421004E4F4950004C494E4B434F15
:10117C004E5452005452415353004652004E4F4C61
:10118C00494E4B00494E490000FF1171FF1176FF8B
:0E119C001180FF1186FF1189FF1190FF119441
:062EB10001430001410095
:102ECD00C2AFC28E758900438910E4F58B758DB83C
:072EDD00D2ABD28ED2AF226E
:03001B000225B704
:1025B700C0E0C083C082C0D0C2AFC28E758B007529
:1025C7008DB8201C0675A61E75A6E10541D218E533
:1025D70043600205430546E546540F7053D223E591
:1025E70046543F7014D21690660CE0600C04F0E07D
:1025F700D394B44004C2AF80FE906607E060020443
:10260700F0E542D3940140021542906104E0600274
:1026170014F090660DE0D394014003E014F0301BF2
:10262700020544E545D394644004D21C8002054565
:10263700E540D3940140021540D28ED2AFD0D0D01E
:0626470082D083D0E032D6
:102D2900E4FFFEFD74DA2DF582E43462F583E02FC9
:102D3900FFE43EFE0DBD10ECE4FD742F2DF582E499
:102D49003461F583E0FC2FFFE43EFEEC60040DBD29
:022D590080E810
:012D5B002255
:10002600C2207D027C007F07122E948F25E5256471
:100036006060097D017F60122E2CD220E4FDFC7FDA
:100046000B122E948F25E52530E6097D04E4FF1278
:100056002E50D2207D017C007F07122E948F25E53D
:10006600257008FD7FFF122E2CD22030200312604F
:1000760000C2AFC288D2A8C2AA1226E2D2AF122DFF
:10008600291213D312264DC21C122C229062D8E0DC
:10009600C3940350037403F0D222D221D220D29308
:1000A6002020077E0F7F6C1221B2E49064F8F012D4
:1000B6002ECDC2AF754201E4A3F0C21DC21ED2AF5F
:1000C60075A70775A61E75A6E1202018AF25FE7D2B
:1000D60003122297E4FF1225097E627FF8E4FB7D76
:1000E6000112237590660CE060037401F0E49061E0
:1000F60004F0A37455F0A37481F0E4F544E4F545E7
:10010600906104E07003122EE490660DE0B40111D4
:100116009080007410F0E490660DF0D220D221D2C7
:1001260022E544D39403402D908002E4F0908001B0
:10013600F0908000F0E544D3940540037401F0E5A7
:1001460044D3940A400FE4F544C2199064F9F0755B
:100156004201122C229080A0E070077FCB7E031212
:1001660029079080B8E07003122A879080D0E0704B
:100176001430241190660374FFF09062CCE0FEA365
:10018600E0FF122B01908000E07013301D10121D4D
:10019600D99062B4EFF0D39400400312071990800F
:1001A60002E07006908000E06005D21B020103C2E7
:1001B6001BE4F544906104E06003020103301F155F
:1001C600121C729062B4EFF0D39400400830170509
:1001D600E0FF122F5A201E030203E2121AF5906264
:1001E600B4EFF0700302010390660CE06003740143
:1001F600F09062F8E054BF247F70030202B61470D8
:10020600030202972402600302038D2020077E0F5B
:100216007F751221B29062D0E0FF70069062D4E042
:100226006055906603E0FEB50722A3E0FF9062D119
:10023600E0B50718906605E0FF9062D2E0B5070CBE
:10024600906606E0FF9062D3E06F602B9062D4E088
:100256006E7035906604E0FF9062D5E0B507299090
:100266006605E0FF9062D6E0B5071D906606E0FFE2
:100276009062D7E0B50711C2199064F97403F012C1
:10028600001E7542010203E290660374FFF002034A
:10029600E29065FBE0FF9062FAE06F60030203E222
:1002A6009065FBE004F0E4F5429064F8F00203E2A6
:1002B6003019030203E29062F9E0D3940A50030274
:1002C6000360A3E0640260030203609062C1E0FF82
:1002D600906303E06F60030201039062C2E0FF9047
:1002E6006304E06F60030201039062C3E0FF906362
:1002F60005E06F60030201039062C4E0FF906306AD
:10030600E06F60030201039062C5E0FF906307E0BF
:100316006F60030201039062C6E0FF906308E06F1E
:1003260060030201037E0F7F831221B29062FB639A
:10033600A2019062B963A2017F12121F2790630D7A
:1003460063A20190660363A2017F04121F279064D3
:10035600F97406F075420202010374C74462700321
:10036600020103122F3FD219E4F5429064F8F0908F
:10037600660704F0E49065FAF0A3F020205E7E0F95
:100386007F8C1221B280553019529062F8E020E736
:100396004B9062FAE0FF9065FAE0FE6F600D9066A2
:1003A60002E07007EE146F703380139065FAE00474
:1003B600F09062B4E0FFD394044003122988906061
:1003C600007482F0A37401F09062FAE0906002F08B
:1003D6007E607F007D03122A0802010320190302B2
:1003E600049E9080D0E0700B9062CCE0FEA3E0FF0C
:1003F600122B01E5427066906607E0D3943C4037C5
:10040600906602E0703112244D9066077401F0E4A4
:100416009063F8F0A37412F09065FBE09063FAF035
:10042600A374FDF090610763A2019063FC63A201CF
:100436007F12121F2780061215B4EF60207E637F9D
:10044600F89063F9E02404FD122A08906602E06041
:10045600030201039062D8E0F542020103122F0A5B
:10046600EF60159060007483F0E4A3F07E607F0077
:100476007D02122A08020103E542640160030201BB
:10048600039064F8E004F0E0C3940540B0C219E4B8
:10049600A3F012001E020103E5426401600302019B
:1004A600039064F9E0147003020542147003020518
:1004B6006E1470030206161470030206CC24FE6046
:1004C6006924066003020103E4F544F52574B025AA
:1004D60025F582E43461F583E0FF74B92525F582BC
:1004E600E43462F583EFF00525E525B43FDF2024EB
:1004F600219062D063A20190660363A2017F041279
:100506001F279064F97401F09064F8F075420302B5
:1005160001039064F97404F09064F87401F0754274
:100526001490660374FFF0020103E4F544122C22D2
:100536009064F97401F0754203020103906603E0CA
:10054600600B9062CCE0FEA3E0FF122B0175420225
:100556009064F97402F09062C7E0700302010390A0
:1005660064F97403F0020103906603E07003020667
:10057600079063F87480F09063FA7402F0E4A3F0D5
:10058600A304F09062C163A2019063FD63A2017FA0
:100596000A121F279064077430F0A3747BF0E4F509
:1005A60025742F2525F582E43461F583E0FF60117B
:1005B60074092525F582E43464F583EFF00525807A
:1005C600E074092525F582E43464F583747DF074BE
:1005D6000A2525F582E43464F583E4F0E525241143
:1005E6009063F9F07C667D039062CCE0FAA3E0FBB1
:1005F6007F021228837E637FF8E5252413FD122AE5
:10060600089064F97404F09062D8E0F542020103A0
:10061600906603E070030206BD9063F87480F09064
:1006260063FA7401F0E4A3F0A304F0A37430F0A31A
:10063600747BF0E4F525742F2525F582E43461F505
:1006460083E0FF601174FF2525F582E43463F583AA
:10065600EFF0052580E074FF2525F582E43463F587
:1006660083747DF074002525F582E43464F583E413
:10067600F0E52524079063F9F07C667D039062CC53
:10068600E0FAA3E0FB7F021228837E637FF8E5256C
:100696002409FD122A08906602E0601B122F3FD241
:1006A60019E4F5429064F8F090660704F0E490656A
:1006B600FAF0A3F00201039064F97404F09062D892
:1006C600E0F542020103906603E0FF6009F460066C
:1006D6009080027410F020242B7542029064F8E09A
:1006E6006401FFF0A37401F0EF60059062D080030F
:1006F6009062D463A20190660363A2017F04121F75
:100706002702010375421490660374FFF002010389
:0207160080FE63
:0107180022BE
:100719009062F9E0B444047F0180027F009062F89E
:10072900E0B447047E0180027E00EE5F604A906279
:10073900C1E09062FAF09062C2E09062FBF09062D0
:10074900C3E09062FCF09062C4E09062FDF09062B8
:10075900C5E09062FEF09062C6E09062FFF09062A0
:10076900F97452F09062AE63A2019080A863A2016D
:100779007F06121F27020C279062B4E0C394085029
:1007890003020C309062C1E0FF9062FAE06F6003EF
:10079900020C309062C2E0FF9062FBE06F600302DE
:1007A9000C309062C3E0FF9062FCE06F6003020CC2
:1007B900309062C4E0FF9062FDE06F6003020C308C
:1007C9009062C5E0FF9062FEE06F6003020C30901A
:1007D90062C6E0FF9062FFE06F6003020C30906632
:1007E9000CE060037401F090660D7464F09062F996
:1007F9007452F09062F8E0644D703C7E0F7F96125F
:1008090021B27E0F7FAC1221B2122C6E7E0F7FD1E6
:100819001221B27E0F7FE11221B27E0F7FED1221EC
:10082900B27E0F7FEF1221B27E0F7FF81221B27EC6
:100839000F7FFA1221B2229062F8E0644C70527E66
:10084900107F471221B2906300E0F526A3E0F52757
:10085900E4F5287D03AF27AE261222977E107F820A
:100869001221B2AE26AF27E4FB7D101223757E0F4D
:100879007FF81221B274102527F527E43526F526CD
:100889000528E528C3941040CA7E0F7FF81221B2CB
:10089900229062F8E0646C705CF52A7E107F851204
:1008A90021B2E4F529AF2A7E007D031222977E103A
:1008B9007F821221B2E4F528A82AE6FF74022528CE
:1008C900F582E43463F583EFF0052A0528E528B4B9
:1008D90010E67E637F02E4FB7D101223757E0F7F95
:1008E900F81221B20529E529C3940840B87E0F7F83
:1008F900F81221B2229062F8E0644B7046F5287430
:10090900EA2528F582E43462F583E0FF6016740075
:100919002528F582E43463F583E0B507100528E559
:1009290028B408DB9061047432F0020C279062F855
:100939007421F0302003020C277E107FC01221B2EF
:10094900020C279062F8E06452704E2020077E1056
:100959007FC81221B2906301E09062B4F0E4F528F7
:100969009062B4E0FDE528C39D5022906300E02524
:100979002824AFF582E43461F583E0FF7402252869
:10098900F582E43463F583EFF0052880D37E627F36
:10099900F8ED240AFD1227FD229062F8E0644970FF
:1009A900452020077E107FD31221B2906300E0F525
:1009B90026A3E0F527E4F528852782852683E0FF2D
:1009C90074022528F582E43463F583EFF00527E501
:1009D90027700205260528E528B480DC7E627FF8A9
:1009E9007D8A1227FD229062F8E064446003020ABE
:1009F90080906300E0FF64447003020C27EFB43178
:100A09000CC2207E107FDB1221B2020C27906300FA
:100A1900E0B4300CD2207E107FE71221B2020C27FD
:100A2900906300E0B4320CD2217E107FF41221B21F
:100A3900020C27906300E0B4330CC2217E117F02BF
:100A49001221B2020C27906300E0B4340CD2227E4A
:100A5900117F111221B2020C27906300E0B4350C0A
:100A6900C2227E117F1E1221B2020C27906300E080
:100A7900FF122F57020C27906104E0701320200702
:100A89007E117F2C1221B29062F87421F0020C279A
:100A99009061047432F09062F8E0FFB45104C2AF7F
:100AA90080FEEF645770452020077E117F3A12219E
:100AB900B2906301E09062B4F0E4F5289062B4E08A
:100AC900FFE528C39F4003020C2774022528F582FD
:100AD900E43463F583E0FF906300E0252824AFF553
:100AE90082E43461F583EFF0052880D09062F8E064
:100AF90064536003020BA22020077E117F45122157
:100B0900B29062C1E0FF9061B8E06F703C9062C240
:100B1900E0FF9061B9E06F70309062C3E0FF9061CF
:100B2900BAE0B507249062C4E0FF9061BBE0B50765
:100B3900189062C5E0FF9061BCE0B5070C9062C6F1
:100B4900E0FF9061BDE06F60169062F87421F030AB
:100B59002003020C277E117F541221B2020C27E4D4
:100B6900F528E4F54574AF2528F582E43461F58369
:100B7900E0FDAF28122D880528E528C394FE40E240
:100B8900C2AFE4907FF0F0A3F0907FFD74AAF0A3C8
:100B990074FFF0A37455F080FE9062F8E0644F7022
:100BA9004B906300E0F526A3E0F527E5274526707D
:100BB9000A2020077E117F5D1221B22020077F2A9B
:100BC9007E001221B2E4F52874022528F582E43466
:100BD90063F583E0852782852683F00527E527705D
:100BE9000205260528E528B480DE80329062F8E007
:100BF900B4452B2020077E117F641221B290630037
:100C0900E0FFA3E0907FF0CFF0A3EFF0C2AF907FB9
:100C1900FD74AAF0A374FFF0A37455F080FE7E6200
:070C29007FF87D081227FD92
:010C300022A1
:102CF100AE07EEC39430400BEED394395005EE2469
:102D0100D0FF22EEC39461400BEED394665005EEE2
:102D110024A9FF22EEC39441400BEED39446500503
:082D2100EE24C9FF22AF0622D7
:1013D300C217E490660CF0D224C21A906602F09011
:1013E30062C163A2019065FC63A2017F06121F27FD
:1013F300E4F526E52675F003A42495F582E434117B
:10140300F583E493FB740193FA740293F91211AA1E
:1014130070030215B3E4F527F528FD742F2DF5822B
:10142300E43461F583E0FF70030215AEE52675F041
:1014330003A42495F582E43411F583E493FB74014A
:1014430093FA740293F98527827583001211C3FE00
:10145300EFB5060875280105270215AAE5287003CC
:101463000215AAEE60030215A5E52624FE602214E8
:101473007003021595147003021599147003021575
:10148300A1240460030215AE90660C7401F00215EA
:10149300AED217742F2DF582E43461F583E0FF6437
:1014A3002D70030215AE122CF1EFC454F0FC74300E
:1014B3002DF582E43461F583E0FF122CF1EF2C90DB
:1014C30065FCF074312DF582E43461F583E0FF129D
:1014D3002CF1EFC454F0FC74322DF582E43461F541
:1014E30083E0FF122CF1EF2C9065FDF074332DF5A2
:1014F30082E43461F583E0FF122CF1EFC454F0FC75
:1015030074342DF582E43461F583E0FF122CF1EF9E
:101513002C9065FEF074352DF582E43461F583E09B
:10152300FF122CF1EFC454F0FC74362DF582E43431
:1015330061F583E0FF122CF1EF2C9065FFF0743717
:101543002DF582E43461F583E0FF122CF1EFC454EE
:10155300F0FC74382DF582E43461F583E0FF122C3E
:10156300F1EF2C906600F074392DF582E43461F5C7
:1015730083E0FF122CF1EFC454F0FC743A2DF58292
:10158300E43461F583E0FF122CF1EF2C906601F057
:101593008019D21A80159066027401F0800DC2245E
:1015A3008009E4F528F5270D02141E05260213F61B
:0115B3002215
:100C31005452414E5A0053545245414D005254535F
:100C41000044454C4159004D4F4445004C494D49E4
:100C510054004556454E504152495459004F444461
:100C6100504152495459004B56545F494E004B561E
:100C7100545F4F555400000A53656E64204B56541F
:100C81003A20000AC1F3F4E5F020E7E0EDFFF2219C
:100C9100000A436865636B73756D206572726F72CC
:100CA100212020000A526563206F6B212020202023
:100CB100202000CCEEE4F3EBFC20EFEEE4E4E5F0E1
:100CC100E6EAE820EEE1ECE5EDE02000F120CAD90A
:100CD1003228332920C1D3D920CAEEECEFE0F1202C
:100CE100F7E5F0E5E720E0E4E0EFF2E5F020D1CE32
:100CF100CC2DC0CCCA0A00F7E5F0E5E720E0F1E829
:100D0100EDF5F0EEEDEDFBE920EFEEF0F22000E283
:100D110020EFE0EAE5F2EDEEEC20F0E5E6E8ECE5C7
:100D21000A00E220EFEEF2EEEAEEE2EEEC20F0E570
:100D3100E6E8ECE50A00CEEFF6E8E820EDE0F1F2B6
:100D4100F0EEE9EAE83A20000A00FF0C31FF0C3727
:100D5100FF0C3EFF0C42FF0C48FF0C4DFF0C53FFF4
:100D61000C5EFF0C68FF0C6FFF0C770011233246FD
:100D71005765748C9DAFBECADBE9F810013322566A
:100D81004775649C8DBFAEDACBF9E8213002136759
:100D9100764455ADBC8E9FEBFAC8D931201203774A
:100DA100665445BDAC9E8FFBEAD8C94253617004BD
:100DB100152736CEDFEDFC8899ABBA52437160142A
:100DC100053726DECFFDEC9889BBAA637240512519
:100DD100340617EFFECCDDA9B88A9B73625041350A
:100DE100241607FFEEDCCDB9A89A8B8495A7B6C26D
:100DF100D3E1F008192B3A4E5F6D7C9485B7A6D2EA
:100E0100C3F1E018093B2A5E4F7D6CA5B48697E3D8
:100E1100F2C0D129380A1B6F7E4C5DB5A49687F3C9
:100E2100E2D0C139281A0B7F6E5C4DC6D7E5F4803C
:100E310091A3B24A5B69780C1D2F3ED6C7F5E490A9
:100E410081B3A25A4B79681C0D3F2EE7F6C4D5A198
:100E5100B082936B7A48592D3C0E1FF7E6D4C5B189
:100E6100A092837B6A58493D2C1E0F0089129B2456
:100E7100AD36BF48C15AD36CE57EF78108931AA5F8
:100E81002CB73EC940DB52ED64FF76028B109926E8
:100E9100AF34BD4AC358D16EE77CF5830A9118A7D8
:100EA1002EB53CCB42D950EF66FD74048D169F20C0
:100EB100A932BB4CC55ED768E17AF3850C971EA1B8
:100EC10028B33ACD44DF56E960FB72068F149D22A8
:100ED100AB30B94EC75CD56AE378F1870E951CA398
:100EE1002AB138CF46DD54EB62F97008811A932C90
:100EF100A53EB740C952DB64ED76FF89009B12AD78
:100F010024BF36C148D35AE56CF77E0A8318912E67
:100F1100A73CB542CB50D966EF74FD8B029910AF57
:100F210026BD34C34AD158E76EF57C0C851E97283F
:100F3100A13AB344CD56DF60E972FB8D049F16A937
:100F410020BB32C54CD75EE168F37A0E871C952A27
:100F5100A338B146CF54DD62EB70F98F069D14AB17
:0B0F610022B930C74ED55CE36AF1787E
:102EB70052660E0000000000000000000000000045
:052EC700000000000006
:032F57008F2B229B
:03002300021FDBDE
:0B1FDB00C0E0C083C082C0D075D018E9
:0B1FE600309862754301AF99300C4940
:101FF100200224301252EF604FEFD39420504974E5
:102001002E250DF582E43467F583EFF0050DD2023C
:1020110025E004F5088031742E250DF582E434673E
:10202100F583EFF0050DD5081F90672CE50DF063E2
:072031000D80530D80C20277
:10203800800F742E250DF582E43467F583EFF005E3
:102048000DC29830996E300369301007309704D26A
:1020580000805F906620E0FFE50EC39F400FC2033B
:10206800D212200B02D214C20BD2968045AF0E05B5
:102078000E742E2FF582E43468F583E0F50F3009ED
:1020880019530F7F30012820D008200422630F80C5
:10209800801D30041A630F808015300112E50F523D
:1020A8000F300406A2D0929B8005A2D0B3929B85E4
:0620B8000F99C299D2AF9E
:0920BE00D0D0D082D083D0E032F2
:022BC9008F2E4D
:102BCB0090672DE0FF04F074212FF582E43466F555
:102BDB00837420F0E4FFEFC39D503BE52E75F003AB
:102BEB00A4244BF582E4340DF583E493FB74019339
:102BFB00FA740293F98F827583001211C3FE9067EA
:102C0B002DE02421F582E43466F583EEF00F906716
:062C1B002DE004F080C072
:012C21002290
:102E0500742F2FF582E43461F583E0FE64206016AB
:102E150090672DE0FD04F074212DF582E43466F50C
:062E250083EEF00F80DADD
:012E2B002284
:10178D00E4F526E52675F003A4244BF582E4340D2B
:10179D00F583E493FB740193FA740293F91211AA81
:1017AD007003021950E4F528F529F527742F252724
:1017BD00F582E43461F583E0FF700302194BE526F1
:1017CD0075F003A4244BF582E4340DF583E493FB0B
:1017DD00740193FA740293F98528827583001211AE
:1017ED00C3FEEFB506087529010528021946E5293E
:1017FD007003021946EE6003021941AD28AF26129F
:10180D002BC9E526B40A00400302194B901820F8A5
:10181D0028287302183E02188A02188F02189402A3
:10182D0018C60218FB02192B0219310219350219BB
:10183D003BAF27122E05742F2527F9E43461FA7B6F
:10184D0001C0031B8B31753200753300E4F534D0C4
:10185D00031219518F2D8E2C8D2B8C2AAB2DAA2C6A
:10186D00A92BA82A7F007E8C7D0A7C0012122C12D7
:10187D0012BE90692EEEF0A3EFF002194BC20C02CE
:10188D00194BD21002194BAF27122E05742F252795
:10189D00F9E43461FA7B01C0031B8B31753200759D
:1018AD003300E4F534D0031219518F2D8E2C8D2B6E
:1018BD008C2AAF2D8F0A02194BAF27122E05742FCC
:1018CD002527F582E43461F583E0B43702D209743B
:1018DD00302527F582E43461F583E0FFB44E04C270
:1018ED00018002D201EF64457054D2048050AF27BD
:1018FD00122E05742F2527F9E43461FA7B01C003FC
:10190D001B8B31753200753300E4F534D003121999
:10191D00518F2D8E2C8D2B8C2A852D098020D20157
:10192D00D204801AD2018016D205D2118010D205B0
:10193D00D20A800AE4F529F52805270217B90526EC
:03194D00021790EE
:011950002274
:10264D00C203C214C208C202C20FE4F50E90662086
:10265D00F0F50AF50DF543C200D297D296C209C224
:10266D0010D20CD21290692E74FFF0A374F4F07591
:10267D000CFFE490672DF075090CC206C213C2055C
:10268D00C20AC21190672B7409F012178DC2ADE406
:10269D00F5C9D2CDD2CCC2C9C2CAF5CDF5CC90699F
:1026AD002EE0F5CBA3E0F5CA85CBCD85CACCE4F5FC
:1026BD009830010C2009095387BFD29FD29E80020A
:1026CD00D29EC2ACC298C29975B81075B710D2CA55
:0526DD00D29CD2AC22EA
:10000600E5116FFF900E6C936510F511EF900D6C76
:0300160093F5104F
:0100190022C4
:032F5A008F26229D
:0220C7008D2763
:1020C900E4F528F511F510AA06A9077B018B2C8ADE
:1020D9002D892E752A68752B301211AAFF333333D7
:1020E90054F890682FF02510F5107401252EF52E5F
:1020F900E4352DF52D7401252EF52EE4352DF52D1C
:10210900E4FFE52724FEFEEFC39E502EAB2C052EDF
:10211900E52EAA2D7002052D14F91211AAFEEF243D
:1021290002FDE433FCED6401242EF58274683CF56C
:1021390083EEF02510F5100F80C8E52704F5283047
:10214900E0020528E528C3131490682EF02510F540
:1021590010F404FEEF2402FDE433FCED6401242EA7
:10216900F58274683CF583EEF00FEF2402FFE43347
:10217900FEEF6401242EF58274683EF583E4F0C213
:1021890002906614E0FCA3E0FDA3E0FEA3E0FFE4F7
:10219900FAF9F8EF2401FFEA3EFEE93DFDE83CFCCF
:0821A9009066141212DDAF284C
:0121B100220B
:10244D00E4FF90672BE0FE7D000FED2407F582E49D
:10245D003461F583EEF00F74072401F582E43461E5
:10246D00F583E4F07C667D13FEED1DAA0470011C5E
:10247D00F5828A83E0FBAA070F74072AF582E434FC
:10248D0061F583EBF00EBE04E07C667D17E4FEED96
:10249D001DAA0470011CF5828A83E0FBAA070F7444
:1024AD00072AF582E43461F583EBF00EBE04E07C7F
:1024BD00667D1BE4FEED1DAA0470011CF5828A8366
:1024CD00E0FBAA070F74072AF582E43461F583EB6C
:1024DD00F00EBE04E07C667D1FE4FEED1DAA0470C7
:1024ED00011CF5828A83E0FBAA070F74072AF58287
:0B24FD00E43461F583EBF00EBE04E058
:0125080022B0
:082F4800C2992099FDD29922E3
:092F3F00D2CAD29CD2ACC2082215
:102CB300AD077E677F211220C7906620EFF0D20315
:102CC300E4F50E2020157E0C7F781221B27E687FFA
:102CD3002E906620E0FDE4FB122375C296301003AC
:0E2CE300D20022E50A6003F54022122F48229B
:102988008F263003087E0C7F841221B2229062FBCE
:10299800E090672BF0300C293005137E627FFAE552
:1029A8002624FCFD1220C7906620EFF0802B7E6263
:1029B8007FFCE52624FCFD1220C7906620EFF080FE
:1029C80018E52624FCFF906620F09062FC63A201C3
:1029D80090682E63A201121F27A211820550057567
:1029E8000B05D213E4F50ED203C296301004D200C0
:1029F800800BE50A6004F5408003122F48C21422B8
:1015B400200603300B037F0022200C030216F39055
:1015C400672CE07003021782FF547FFEE49063F8F7
:1015D400F0A3EEF09065FBE09063FAF0A37416F0CC
:1015E4007526637527FCE4F510EF5480FF242FF56E
:1015F40082E43467F583E02510F510131313541FA8
:10160400FD0527E527AA267002052614F5828A839C
:10161400EDF0742E2FF582E43467F583E0FF05279F
:10162400E527AC267002052614F5828C83EFF0259D
:1016340010F510E4FFEE24FEFDEFC39D502DEF24C2
:1016440002FDE433FCED6401242EF58274673CF55D
:1016540083E0FD0527E527AA267002052614F582F6
:101664008A83EDF02510F5100F80CAE510605190C3
:101674006618E0FCA3E0FDA3E0FEA3E0FFE4FAF9B2
:10168400F8EF2401FFEA3EFEE93DFDE83CFC9066EC
:10169400181212DD2020217E0C7F921221B2906755
:1016A4002CE0FD5480242EF582E43467AF82FEEDF5
:1016B400547FFDE4FB122375E490672CF00217823B
:1016C400906610E0FCA3E0FDA3E0FEA3E0FFE4FAD3
:1016D400F9F8EF2401FFEA3EFEE93DFDE83CFC9009
:1016E40066101212DDE490672CF0D215021782E521
:1016F4000D547FFFD394005003021782E543D39423
:10170400055006EFC395094075C2AF90672CE50DEF
:10171400F0630D80530D80E4F543C202C208D2AFDA
:101724009063F8F090672CE0FE547FFF9063F9F02B
:101734009065FBE09063FAF090672BE09063FBF018
:10174400EE5480242EF582E43467F58363A201907D
:1017540063FC63A201121F272020217E0C7FA512A7
:1017640021B290672CE0FD5480242EF582E4346786
:10177400AF82FEED547FFDE4FB122375D2153015C4
:0817840005C2157F01227F0060
:01178C00223A
:102C6E007E0C7FB41221B27E0C7FCD1221B27E0C6F
:102C7E007FF81221B2300C097E0D7F101221B28026
:102C8E00077E0D7F231221B27E0D7F371221B27E79
:102C9E00667F2190672DE0FD7B051223757E0D7FEB
:052CAE00491221B222D1
:05001E00C2AEC2AC22DD
:102EE400300008209705C200122F48E540B40106BF
:072EF400E4F540122F482213
:0E2F0A00301408201305C2147F01227F00221C
:03000300022B6865
:0D2B6800C0E0C083C082C0D075D000C0079F
:102B7500C2A8908008E0FFEF54F06035EF30E4081C
:102B8500D21D9080087410F0EF30E508D21F9080B8
:102B9500087420F0EF30E608D21E9080087440F0EB
:102BA500EF30E7069080087480F0908008E0FF80A1
:092BB500C690800874FFF0D2A85C
:0B2BBE00D007D0D0D082D083D0E0320E
:102C22009080007480F09062B963A201F583F5820E
:102C320063A2017F08121F279062C163A2019080E4
:102C42008863A2017F0A121F279062CBE0FF908067
:102C5200B1F09080E1EFF09080957455F0A3F09080
:0C2C620080007401F09080097470F02272
:04290700AD07AC0666
:10290B00908009E04410F09080A0E0706F9080A15F
:10291B007482F09080A874FFF0A3F0A3F0A3F0AF43
:10292B0004AE079080AEEEF0AE05A3EEF0AE0790CE
:10293B0080ACEEF0AE05A3EEF09080007402F09048
:10294B0069301212E900000000906930E09080407D
:10295B00F0906931E0908041F0906932E0908042D4
:10296B00F0906933E0908043F0A3E4F0A3F0A3F080
:0C297B00A3F0908018F0A3F0A3F0A3F0EC
:01298700222D
:042B0100AD07AC066A
:102B0500908009E04440F09080D0E070559080D1ED
:102B15007482F0AF049080DEEFF0AF05A3EFF09084
:102B250080027402F09069341212E90000000090EE
:102B35006934E0908058F0906935E0908059F090C4
:102B45006936E090805AF0906937E090805BF0A399
:102B5500E4F0A3F0A3F0A3F0908030F0A3F0A3F08D
:022B6500A3F0DB
:012B6700224B
:102A8700908009E04420F09080B8E0706C9080B9A5
:102A97007482F07F039080C6EFF07FCDA3EFF07FC5
:102AA700039080C4EFF0A374CDF09080C074FFF062
:102AB700A3F0A3F0A3F09080017402F0906938129C
:102AC70012E900000000906934E090804CF09069B2
:102AD70035E090804DF0906936E090804EF0906937
:102AE70037E090804FF0A3E4F0A3F0A3F0A3F090B9
:092AF7008024F0A3F0A3F0A3F089
:012B000022B2
:102883008C268D27A907EAFDE975F018A424ACFF6F
:10289300E5F034808F82F583EDF0EBFDE975F018F8
:1028A300A4FFAEF024ACFBEE34808B82F583A3ED62
:1028B300F08527828C83E0FDEF24A8FFEE3480FEB1
:1028C3008F82F583EDF08527828C83A3E08F828E40
:1028D30083A3F0852782852683A3A3E0FDE975F012
:1028E30018A424A8FFE5F03480FE8F82F583A3A308
:1028F300EDF08527828C83A3A3A3E08F828E83A32D
:04290300A3A3F02278
:0627FD008D2BAB07AA06BC
:10280300906930E0FCA3E0FDA3E0FEA3E0F52F8E8A
:102813002E8D2D8C2CAE02AF038E838F8263A2018B
:10282300E52E540744C0F583852F8263A201AF2BA5
:10283300121F6D908000E020E5F9E4FCFDFEE52F1A
:10284300252BF52FEE352EF52EED352DF52DEC350B
:102853002CF52CC2A8908040E52CF0A3E52DF0A325
:10286300E52EF0A3E52FF0D2A89080007420F0AFFE
:0F2873002FAE2EAD2DAC2C9069301212DDAF2B95
:012882002233
:062A08008D26AB07AA06B3
:102A0E00906934E0FCA3E0FDA3E0FEA3E0F52A8E7E
:102A1E00298D288C27AE02AF038E838F8263A2018D
:102A2E00E529540744D0F583852A8263A201AF2697
:102A3E00121F6DE4FCFDFEE52A2526F52AEE35294A
:102A4E00F529ED3528F528EC3527F527C2A8908015
:102A5E0058E527F0A3E528F0A3E529F0A3E52AF031
:102A6E00D2A89080027420F0AF2AAE29AD28AC27F0
:082A7E009069341212DDAF264D
:012A8600222D
:022509008F261B
:10250B00908001E030E5037F0022906938E0FCA366
:10251B00E0FDA3E0FEA3E0F52A8E298D288C279001
:10252B0065FC63A201E529540744C8F583852A821B
:10253B0063A2017F06121F83E52A2406F52AE435E0
:10254B0029F529E43528F528E43527F5279064FA91
:10255B0063A201E529540744C8F583852A8263A247
:10256B0001AF26121F83E4FCFDFEE52A2526F52A82
:10257B00EE3529F529ED3528F528EC3527F527C259
:10258B00A890804CE527F0A3E528F0A3E529F0A35C
:10259B00E52AF0D2A89080017420F0AF2AAE29ADC5
:0B25AB0028AC279069381212DDAF2623
:0125B6002202
:101DD900C2A89081E0E0F5260526052605260526F8
:101DE900052605260526052605260526908010E0E8
:101DF900F529A3E0F52AA3E0F52BA3E0F52C9081C2
:101E0900E1E0F526052605260526052605260526EB
:101E19000526052605260526908014E0F52DA3E064
:101E2900F52EA3E0F52FA3E0F530D2A8E52FB52BC9
:101E390008E530B52C037F0022E4F526E52F540789
:101E490044E0F58385308263A2019062F863A201C0
:101E59007F08121F9B9062FA63A2019062AE63A28F
:101E6900017F06121F279062F8E0F527A3E0F52805
:101E7900E4F5269062F8E0702AA3E024F8F526E557
:101E89002F540744E0F58385308274082582F58252
:101E9900E43583F58363A2019062F863A201AF265A
:101EA900121F9BAE27E4FCFDE5302528F530E52F10
:101EB9003EF52FED352EF52EEC352DF52DC2A890DA
:101EC9008014E52DF0A3E52EF0A3E52FF0A3E5306E
:0B1ED900F0D2A89080007440F0AF260B
:011EE40022DB
:101AF500C2A89081E6E0F5260526052605260526D9
:101B0500052605260526052605260526908028E0B6
:101B1500F529A3E0F52AA3E0F52BA3E0F52C9081A8
:101B2500E7E0F526052605260526052605260526CC
:101B3500052605260526052690802CE0F52DA3E033
:101B4500F52EA3E0F52FA3E0F530D2A8E4F526E5C0
:101B55002FB52B0AE530B52C05C21E021C53E52F07
:101B6500540744F0F58385308263A2019062F863DF
:101B7500A2017F08121F9B9062F8E0F527A3E0F50C
:101B850028E528452770099080027410F07F00220F
:101B9500906603E0FFF4602D9062FAE06F70769036
:101BA5006604E0FF9062FBE06F706A906605E0FFF7
:101BB5009062FCE06F705E906606E0FF9062FDE06B
:101BC5006F602280509062FAE0906603F09062FBAD
:101BD500E0906604F09062FCE0906605F09062FD8E
:101BE500E0906606F09062F8E0702AA3E024F8F52C
:101BF50026E52F540744F0F5838530827408258245
:101C0500F582E43583F58363A2019062F863A2014E
:101C1500AF26121F9BAE27E4FCFDE5302528F530E5
:101C2500E52F3EF52FED352EF52EEC352DF52DAFA7
:101C35002CAE2BAD2AAC29AB30AA2FA92EA82DD3BB
:101C45001212CC40099080027410F07F0022C2A8C5
:101C550090802CE52DF0A3E52EF0A3E52FF0A3E56C
:0C1C650030F0D2A89080027440F0AF264E
:011C71002250
:101C7200C2A89081E3E0F52605260526052605265D
:101C820005260526052605260526052690801CE044
:101C9200F529A3E0F52AA3E0F52BA3E0F52C90812A
:101CA200E4E0F52605260526052605260526052651
:101CB2000526052605260526908020E0F52DA3E0C1
:101CC200F52EA3E0F52FA3E0F530D2A8E4F526E542
:101CD2002FB52B0AE530B52C05C21F021DBAE52F20
:101CE200540744E8F58385308263A201906004635F
:101CF200A2017F0E121FB1906004E0F527A3E0F568
:101D0200289065FCE0FF90600CE06F706C9065FDC0
:101D1200E0FF90600DE06F70609065FEE0FF906004
:101D22000EE06F70549065FFE0FF90600FE06F70FF
:101D320048906600E0FF906010E06F703C90660192
:101D4200E0FF906011E06F7030906004E0702AA3B1
:101D5200E024F2F526E52F540744E8F58385308226
:101D6200740E2582F582E43583F58363A2019060C7
:101D72000463A201AF26121FB1AE27E4FCFDE530D9
:101D82002528F530E52F3EF52FED352EF52EEC35D5
:101D92002DF52DAF2CAE2BAD2AAC29AB30AA2FA935
:101DA2002EA82DD31212CC5006E528452770099093
:101DB20080017410F07F0022C2A8908020E52DF0EF
:101DC200A3E52EF0A3E52FF0A3E530F0D2A8908092
:061DD200017440F0AF2691
:011DD80022E8
:0421B2008E2B8F2CB5
:1021B600906930E0FCA3E0FDA3E0FEA3E0F5328EDB
:1021C600318D308C2FE532FFE5315407FEE42FF5D3
:1021D6002EEE34C0F52D852E82F5837423F0052E60
:1021E600E52E7002052D532DC7F582852D83740AC1
:1021F600F0052EE52E7002052D532DC79062C163A2
:10220600A201852D83852E8263A2017F06121F6D92
:102216007406252EF52EE4352DF52D852B83852C7C
:102226008263A201852D83852E8263A201121F512E
:10223600908000E020E5F9E4FCFDFE906930E0F8CE
:10224600A3E0F9A3E0FAA3E02FFFEE3AFEED39FD95
:10225600EC38FCEF2408FFE43EFEE43DFDE43CFCE4
:102266009069301212DDC2A8906930E0908040F08B
:10227600906931E0908041F0906932E0908042F0C0
:10228600906933E0908043F0D2A89080007420F0EB
:012296002225
:062375008E2B8F2C8D2D34
:10237B00906930E0FCA3E0FDA3E0FEA3E0F5338E13
:10238B00328D318C30E533FFE5325407FEE42FF507
:10239B002FEE34C0F52E852F82F5837423F0052F95
:1023AB00E52F7002052E532EC7F582852E83EBF099
:1023BB00052FE52F7002052E532EC79062C163A225
:1023CB0001852E83852F8263A2017F06121F6D74F8
:1023DB0006252FF52FE4352EF52E852B83852C82A4
:1023EB0063A201852E83852F8263A201AF2D121F5D
:1023FB006D908000E020E5F97408252DF52DFFE4A4
:10240B00FCFDFEE5332FF533EE3532F532ED35318C
:10241B00F531EC3530F530C2A8908040E530F0A3B3
:10242B00E531F0A3E532F0A3E533F0D2A8908000BC
:10243B007420F0AF33AE32AD31AC30906930121244
:01244B00DDB3
:01244C00226D
:062297008E2B8F2CAB051D
:10229D00906930E0FCA3E0FDA3E0FEA3E0F5328EF3
:1022AD00318D308C2FE532FFE5315407FEE42FF5EB
:1022BD002EEE34C0F52D852E82F5837423F0052E78
:1022CD00E52E7002052D532DC7F582852D83EBF07C
:1022DD00052EE52E7002052D9062C163A201852D9C
:1022ED0083852E8263A2017F06121F6D7406252E33
:1022FD00F52EE4352DF52D532DC7E52B852E828535
:10230D002D83F0052EE52E7002052D532DC7F58278
:10231D00852D83E52CF0052EE52E7002052D532D10
:10232D00C7908000E020E5F9E532240AF532E43566
:10233D0031F531E43530F530E4352FF52FC2A89065
:10234D008040E52FF0A3E530F0A3E531F0A3E532B1
:10235D00F0D2A89080007420F0AF32AE31AD30AC29
:07236D002F9069301212DD10
:012374002246
:1026E200E4F526E52604FF122DB274B92526F582FB
:1026F200E43462F583EFF00526E526C3943F40E318
:10270200E4F526E526247FFF122DB2742F2526F547
:1027120082E43461F583EFF0742F2526F582E434E8
:1027220061F583E0701D742F2526F582E43461F58E
:10273200837420F074302526F582E43461F583E455
:10274200F080090526E526C3948040B7E49061AE87
:10275200F0F526AF26122DB274AF2526F582E434A9
:0E27620061F583EFF00526E526C394FE40E501
:012770002246
:102E7400E4FDFCC3ED9FEC9E5015E4FBFA0BBB0094
:0F2E8400010ABA01F8BB90F50DBD00010C80E406
:012E9300221C
:0D2F18004390014390025390FE5390FD2220
:0D2F25005390FD5390FE4390024390012213
:0E2EFB005390FD439002E5905408FF5390FD64
:012F090022A5
:0D2F32005390FD4390014390025390FD2207
:072F5000AE071FEE70FA222C
:022D5C00AD07C1
:102D5E00E4FC5390FDEDA804088002C333D8FC3088
:102D6E00E70543900180035390FE7F05122F5043D9
:092D7E0090020CBC08DC5390FD2E
:012D87002229
:102DDC00E4FF5390FD7E07439002E59030E00D74C4
:102DEC0001A806088002C333D8FC42075390FD1E8D
:082DFC00C3EE6480948050DFF7
:012E040022AB
:102D8800AB05AA07122F187FA0122D5C122EFBAFDD
:102D980002122D5C122EFBAF03122D5C122EFB12B9
:0A2DA8002F257F0A7E00122E7422F0
:022DB200AB076D
:102DB400122F187FA0122D5C122EFBAF03122D5C74
:102DC400122EFB122F187FA1122D5C122EFB122D36
:072DD400DC122F32122F2543
:012DDB0022D5
:102E9400A2AF9225C2AF8C838D82EF121FC943A2C9
:0C2EA40020121FCB53A2DFA22592AFFF2B
:012EB00022FF
:022E2C008F26EF
:102E2E00A2AF9225C2AFE4F5838D827406121FC93C
:102E3E00E52643A220121FCB53A2DFA22592AF7F1D
:012E4E000182
:012E4F002260
:022E50008F26CB
:102E5200A2AF9225C2AFE4F5838D82740A121FC914
:102E6200E52643A220121FCB53A2DFA22592AF7FF9
:012E7200015E
:012E7300223C
:101EE500740093F8ECC3984024701F740193F8EDC7
:101EF500C39840197014740293F8EEC398400E709D
:101F050009740393F8EFC39840037F00227F0122F1
:101F1500EDF8E6F008A3DFFA22EDF8E0F608A3DF16
:101F2500FA22E0A363A201F0A363A201DFF475A284
:101F35000022E0A363A2016DFE936CFDEE05839381
:101F4500FC158363A201DFEA75A200227F00E493FA
:101F5500A363A201F00F600CA3E583C2E3F58363DD
:101F6500A20180EA75A20022E0A363A201F0A3E525
:101F750083C2E3F58363A201DFEE75A20022E0A32D
:101F850063A201F0A3E583C2E4D2E3F58363A20172
:101F9500DFEC75A20022E583C2E3F583E0A363A22B
:101FA50001F0A363A201DFEE75A20022E583C2E47E
:101FB500D2E3F583E0A363A201F0A363A201DFEC02
:0F1FC50075A20022F922C002C004C00612FFF06C
:071FD400D006D004D0022268
:10277D00020026E493A3F8E493A34003F68001F24C
:10278D0008DFF48029E493A3F85407240CC8C3335D
:10279D00C4540F4420C8834004F456800146F6DF2C
:1027AD00E4800B0102040810204080902EB1E47EDD
:1027BD00019360BCA3FF543F30E509541FFEE49321
:1027CD00A360010ECF54C025E060A840B8E493A3E8
:1027DD00FAE493A3F8E493A3C8C582C8CAC583CA13
:1027ED00F0A3C8C582C8CAC583CADFE9DEE780BECB
:012ECC000005
:1011AA00BB010689828A83E0225002E722BBFE0243
:0911BA00E32289828A83E4932276
:1011C300BB010CE58229F582E5833AF583E02250E1
:1011D30006E92582F8E622BBFE06E92582F8E2222B
:0D11E300E58229F582E5833AF583E4932245
:1011F00075F008758200EF2FFFEE33FECD33CDCCB6
:1012000033CCC58233C5829BED9AEC99E582984038
:101210000CF582EE9BFEED9AFDEC99FC0FD5F0D615
:10122000E4CEFBE4CDFAE4CCF9A88222B800C1B93F
:101230000059BA002DEC8BF084CFCECDFCE5F0CB7D
:10124000F97818EF2FFFEE33FEED33FDEC33FCEBB6
:1012500033FB10D703994004EB99FB0FD8E5E4F971
:10126000FA227818EF2FFFEE33FEED33FDEC33FC5E
:10127000C933C910D7059BE99A4007EC9BFCE99A52
:10128000F90FD8E0E4C9FAE4CCFB2275F010EF2F97
:10129000FFEE33FEED33FDCC33CCC833C810D70797
:1012A0009BEC9AE899400AED9BFDEC9AFCE899F8D2
:0E12B0000FD5F0DAE4CDFBE4CCFAE4C8F92265
:0E12BE00C3E49FFFE49EFEE49DFDE49CFC2241
:1012CC00EB9FF5F0EA9E42F0E99D42F0E89C45F078
:0112DC0022EF
:0C12DD00ECF0A3EDF0A3EEF0A3EFF02284
:1012E900A8828583F0D083D08212130012130012D2
:1012F9001300121300E473E493A3C583C5F0C583F7
:10130900C8C582C8F0A3C583C5F0C583C8C582C84E
:0113190022B1
:101951008B2E8A2F8930E4F53AF539F538F537F5CC
:1019610035F536E532453345316012EBC0E0EAC06A
:10197100E0E9C0E0AB31AA32A933121369AB2E05FD
:1019810030E530AA2F7002052F14F91211AAF53B88
:10199100C394094007E53BD3940D40E1E53B642046
:1019A10060DBE53BB42D054336038016E53BB42BE4
:1019B10005433601800C74FF2530F53074FF352F57
:1019C100F52FE53460046410703FAB2EAA2FA930C7
:1019D1001211AA64306009E534702E75340A802929
:1019E1009000011211C3FF64786004EFB4581343EF
:1019F100360175341074022530F530E4352FF52F9A
:101A01008007E5347003753408AB2E0530E530AA44
:101A11002F7002052F14F91211AAF53BC3946140EE
:101A21000AE53BD3947A5003533BDF74D0253BF551
:101A31003BC3940A400CE53B9411406D74F9253B7E
:101A4100F53BE53BD395345060433601853A3F85FC
:101A5100393E85383D85373CAF347E00E4FCFDAB33
:101A61003AAA39A938A83712131AC8ECC8C9EDC95E
:101A7100CAEECACBEFCBE4FCFDFEEB253BF53AEE1B
:101A81003AF539ED39F538EC38F537AF3AAE39ADCD
:101A910038FCAB3FAA3EA93DA83CD31212CC50035F
:101AA100021A0A433604021A0AE53620E003E480EA
:101AB1002DE53245334531601EAB2EE53024FFF96B
:101AC100E52F34FFFAEBC0E0EAC0E0E9C0E0AB315A
:101AD100AA32A933121369E53630E20774FFFFFE1B
:101AE100FDFC22E536AF3AAE39AD38AC3730E10313
:041AF1000212BE22FD
:10131A00E88FF0A4CC8BF0A42CFCE98EF0A42CFC72
:10132A008AF0EDA42CFCEA8EF0A4CDA8F08BF0A4F0
:10133A002DCC3825F0FDE98FF0A42CCD35F0FCEB4F
:10134A008EF0A4FEA9F0EB8FF0A4CFC5F02ECD3914
:0F135A00FEE43CFCEAA42DCE35F0FDE43CFC2281
:10136900BB011A89828A83D0F0D0E0F8D0E0F9D0A5
:10137900E0FAD0E0FBE8C0E0C0F00213C15016E982
:10138900F8D083D082D0E0F9D0E0FAD0E0FBC08277
:10139900C0830213B8BBFE16E9F8D083D082D0E02F
:0F13A900F9D0E0FAD0E0FBC082C0830213CA2261
:0913B800EBF608EAF608E9F6225A
:0913C100EBF0A3EAF0A3E9F0222D
:0913CA00EBF208EAF208E9F22254
:00000001FF
